:020000020000fc
:040000000001703a51
:0400010004c00074c3
:040002009801483adf
:040003009cfff80462
:04000400983ffd1e06
:040005000000203a9d
:04000600002ee03aae
:0400070000001006df
:04000800017fffc4b1
:04000900002ee03aab
:04000a0000004306a9
:04000b003007883af8
:04000c00002ee03aa8
:04000d0000004006a9
:04000e003009883af3
:04000f0018000426ab
:04001000197fff262f
:04001100002ee03aa3
:040012000000520692
:04001300003ff506af
:04001400002ee03aa0
:0400150000003206af
:04001600203ee83a66
:04001700003fff06a1
:04001800bb400104e4
:04001900001ce03aad
:04001a0074807fd49b
:04001b009480004489
:04001c00008000045c
:04001d00002ee03a97
:04001e0000002406b4
:04001f0004010004d4
:0400200003c0158480
:0400210003803fc455
:04002200002ee03a92
:04002300000036069d
:0400240053c0062699
:040025005380181ece
:04002600843fffc450
:04002700803ffa1efe
:04002800002ee03a8c
:0400290000001e06af
:04002a00003fff068e
:04002b00002ee03a89
:04002c0000002106a9
:04002d00002ee03a87
:04002e0000001f06a9
:04002f003005883ad6
:040030000443c3f4ce
:040031008c43c3c475
:0400320004000104c1
:04003300145c703aaf
:04003400741c983a66
:040035001404d83a9d
:040036001444703ac4
:040037001384b03a44
:040038008020d07ada
:040039008c1c983a49
:04003a008ba2f03a6b
:04003b00803ff71eed
:04003c00108001c46b
:04003d001004d0fae1
:04003e00002ee03a76
:04003f0000000806af
:04004000002ee03a74
:0400410000000106b4
:040042006800683ab0
:0400430003010004b1
:0400440093000335ed
:0400450002c0c03401
:040046005896b03ade
:0400470000000706a8
:04004800bdc0010432
:0400490093000237e7
:04004a006300080c3b
:04004b00603ffd26ef
:04004c0090000335e8
:04004d00b800683a55
:04004e000017883ad5
:04004f00ba000104ee
:04005000000d883add
:0400510005000104a1
:040052005816123af0
:04005300002ee03a61
:04005400000006069c
:04005500328cb03aff
:04005600300c163a1a
:04005700a53fffc4fe
:04005800a03ff91eae
:040059004000683ac1
:04005a000017883ac9
:04005b00bdc001041f
:04005c009240023795
:04005d004a40100cf9
:04005e00483ffd26f4
:04005f0092c0013515
:040060009240023791
:040061004a40200ce5
:04006200483ffd26f0
:040063009280002364
:04006400b800683a3e
:04006500bdc0010415
:040066001907883ab4
:0400670018ffffc4bb
:040068009240023789
:040069004a40100ced
:04006a00483ffd26e8
:04006b0090000135cb
:04006c009240023785
:04006d004a40200cd9
:04006e00483ffd26e4
:04006f009240003784
:0400700090000135c6
:040071002240002504
:040072002100004425
:0400730020fff81e54
:04007400924002377d
:040075004a40200cd1
:04007600483ffd26dc
:04007700924000377c
:0400780022400025fd
:04007900b800683a29
:04007a000000000082
:04007b000000000081
:04007c000000000080
:04007d00000000007f
:04007e00000000007e
:04007f00000000007d
:00000001FF
